:04000000B401EB2834
:10000800F000030E8301BC000A08B70000308A0024
:10001800F2280408A700091009118910831609108D
:1000280009118910860183122708B41836283A3036
:10003800A1009830A1203330A60049201330A10038
:100048008830A12049206430A02049206430A020B5
:10005800383035200C30352006303520B4142708C8
:1000680036283414A600341C44280911033C031C08
:10007800492849201330A1008830A1200314080022
:100088003414FE3C0319E6280915091426088600CD
:1000980000004E2834100910C830A02003140800AE
:1000A800B61329080319B6170530A8002730A3008E
:1000B80010306A200330A300E8306A20A3016430BE
:1000C8006A20A3010A306A2024087128A2002508A2
:1000D800A1002408A000C5202008A000A803031937
:1000E800B613290803197B282802031808002008DA
:1000F800031DB613B61B0800303EE128A000A00D72
:10010800A00D200D3839C1389F000030A1003230D1
:10011800A1201F151F198E28A1011E08E628A3017A
:10012800A200FF30A207031CA307031CE628033024
:10013800A100E630A1209528A101FC3EA000A1095C
:100148000000031CAD28FF30A928A0070318A82821
:10015800A0076400AF28A10FA7280800A301A200E8
:100168000530A80023082102031DBC28220820020C
:10017800043003180130031902302805031DFF302D
:10018800E628A501A4011030A600210DA40DA50D97
:100198002208A4022308031C230FA5020318DB2846
:1001A8002208A40723080318230FA5070310A00D8E
:1001B800A10DA60BC9282008E628840031088A006A
:1001C80030088200831303138312640008000710A9
:1001D8008316071083128A110A12BD290408B50074
:1001E80019308A008C193A218301350884003708B0
:1001F8008A003C0E8300F00E700E09003D3084002A
:1002080008308A150A1678208A01E6208A110A120F
:10021800031C022908003D3084008A150A160020B4
:100228008A01E6208A110A12031C0F29CE00080051
:100238008316FF30850002309F0083120800831662
:1002480007309F0083120508D700831602309F00ED
:1002580083120800831606088312D8008316FF301D
:10026800860083120608D700580883168600831272
:100278000800831686018312570886000800831633
:1002880007088312D8008316FF30870083120708F7
:10029800D700580883168700831208008316870141
:1002A8008312570887000800831608088312D800AD
:1002B8008316FF30880083120808D7005808831671
:1002C8008800831208008316880183125708880063
:1002D8000800831609088312D8008316FF308900A6
:1002E80083120908D700580883168900831208006A
:1002F8008316890183125708890008003E08043CC8
:100308008A110A12031C98298A110A128F21CD001A
:100318008A110A12982901308A003E08820741345E
:100328004234433444344534FE308A010E200130CF
:100338008A010E2050308A010E206F308A010E206B
:1003480072308A010E2074308A010E203A308A01F8
:100358000E204D088A010E203D308A010E20A90189
:100368003F08A400A5010D30B000B1018A01542056
:1003780008000830CE008A011C21071083160710D8
:10038800103083128A01A0208A150A1619216400E8
:100398008316031717080339033A8A110A128312BE
:1003A8000313031DCB29071483160710FE3083128D
:1003B8008A010E2001308A010E2055308A010E2054
:1003C80053308A010E2042308A010E2020308A01E3
:1003D8000E2052308A010E2065308A010E206130CD
:1003E8008A010E2064308A010E2079308A010E209D
:1003F8003D3084008A150A1600208A01E6208A11F9
:100408000A12031CFC29CE0064003D08003C8A1136
:100418000A12031DAA2A64003E08003C8A110A1227
:10042800031D1F2AFE308A010E2001308A010E208A
:100438008A110A12A72AD0016400043050028A11D6
:100448000A120318A72A5008033C8A110A12031C2F
:100458003C2A8A110A123422D5008A110A123C2A2F
:1004680002308A00500882070134C0349434D434EE
:1004780001305007B200B301B30D3208A0003308B1
:10048800A1003F088A01B2208A110A12031DA22A7C
:10049800400AD400FE308A010E2055088A010E2039
:1004A8000430D1006400083051028A110A1203187E
:1004B8006A2A51083D3E84000008B20032088A01C9
:1004C8000E20D10A8A110A12031D562A0430D300BD
:1004D8006400540853028A110A120318A22A8A01D6
:1004E8000F2164003D08003C8A110A12031D7F2A6F
:1004F8008A110A12A22A0130D10064000830510280
:100508008A110A120318A02AD30A64005308540255
:100518008A110A12031D932A8A110A12A22A510863
:100528003D3E84000008B20032088A010E20D10A3C
:100538008A110A12031D812A8A01732AD00A8A1194
:100548000A12031D202A8A110A12C42B64003D08CE
:10055800013C8A110A12031DEC2A64003E08003C83
:100568008A110A12031DBA2A8A01232164003E084F
:10057800013C8A110A12031DC32A8A012E21640034
:100588003E08023C8A110A12031DCC2A8A01432123
:1005980064003E08033C8A110A12031DD52A8A0109
:1005A800582164003E08043C8A110A12031DDE2A01
:1005B8008A016D215708BF0064004008013C8A1178
:1005C8000A12031DE92A8A0182218A110A12C42B00
:1005D80064003D08023C8A110A12031D352B640091
:1005E8003E08013C8A110A12031D002B3F08D70060
:1005F8008A013D218A012E2164003E08023C8A11AD
:100608000A12031D0D2B3F08D7008A0152218A01C7
:10061800432164003E08033C8A110A12031D1A2B69
:100628003F08D7008A0167218A01582164003E08E3
:10063800043C8A110A12031D272B3F08D7008A01A0
:100648007C218A016D215708BF0064004008013CE5
:100658008A110A12031D322B8A0182218A110A1279
:10066800C42B64003D08033C8A110A12031D702B39
:1006780000308A018220C70032308A01932001307D
:100688008A018220C80032308A01932002308A0110
:100698008220C90032308A01932003308A018220E7
:1006A800CA0032308A01932004308A018220CB00AC
:1006B80032308A0193200130BD004708BE00480847
:1006C800BF004908C0004A08C1004B08C200C30166
:1006D800C4018A110A12C42B64003D08043C8A1123
:1006E8000A12031DA92BCF01640007304F028A119B
:1006F8000A120318A62B4F08063C8A110A12031C7B
:10070800972B8A110A128C23CD008A110A12972B73
:1007180003308A004F088207413443345434493443
:1007280056344534213401304F07B200B301B30DBC
:1007380032083D3E84004D088000CF0A8A110A1213
:10074800031D782B8A110A12C42BFE308A010E2051
:10075800C0308A010E2057308A010E2061308A018C
:100768000E2069308A010E2074308A010E2069300B
:100778008A010E206E308A010E2067308A010E2011
:0E0788008A0102218A01FC2963008A01C82B24
:10300000030883120317CC000408C30083160317B8
:10301000A81B3628290883120317C200C100031910
:103020002628831603172A0883120317CD00831757
:103030004D0884000008F20043088400CC1F83136D
:1030400072088000C30ACD0AC20B1728831628080D
:103050004039403A8838A8000830A9008312410856
:10306000F2004C088300720803140800831203174F
:103070004C08830003100800030883120317CC00D8
:103080000408C30083160317B01B7228310883128B
:103090000317C200C1000319622883160317320800
:1030A00083120317CD0083174D0884000008F20037
:1030B00043088400CC1F831372088000C30ACD0A22
:1030C000C20B5328831630084039403A8838B00084
:1030D0000830B10083124108F2004C0883007208E6
:1030E00003140800831203174C0883000310080020
:1030F000F200030883120317CC0072080F39C200D4
:103100000408CD00420883160317AC1BA928AD00A4
:1031100003199D282E088312C3008317CC1F831325
:103120004D0884000008F2008317430884007208E9
:103130008000C30ACD0AC20B8D2883162C084039A3
:10314000403A8838AC00831203174C0883000314FC
:10315000080003100800F200030883120317CC00D4
:1031600072080F39C2000408CD0042088316031705
:10317000B41BDC28B5000319D02836088312C3001D
:103180008317CC1F83134D0884000008F2008317B7
:103190004308840072088000C30ACD0AC20BC0280D
:1031A000831634084039403A8838B4008312031734
:1031B0004C08830003140800031008008317033928
:1031C000983E84000014080083170339983E840059
:1031D0000010080083120317491CF92883161011E8
:1031E000111595146300000095101012111610119E
:1031F0001111080083120317D21C0C29C801B0302A
:10320000CA00831615158312C80F0429CA0F042992
:10321000831615118312D210080083160317951117
:103220008312CA01C801C80F1329CA0F1329192113
:1032300008008316031797010130910090010830B0
:1032400095008312D0010130D200AB01AC01AD0179
:10325000FF30D100831203138C1183168C150B17CA
:103260008B17080083160317951195149701031304
:103270008C11080083160317100811058312031917
:103280005129D500D519A2218312031755185521AC
:10329000D51A8721D5188E21551A7B2155199721CA
:1032A0003A29831203138C110800D001C901831637
:1032B00090119011901190118830A000B830A200A8
:1032C0000830A1000830A400C030A600960190018B
:1032D000831203138C1183160317063098003B30BA
:1032E0009100FF3093000130970083120030D2002C
:1032F0000313031708008316111210121111101175
:10330000831203138C1183120317491408008316C8
:103310009012831203138C11031708008316901068
:10332000831203138C1103178312031708008316EB
:103330001111101111121012831203138C110317A3
:10334000C90108008317831603171408A03E8400E0
:1033500083120008A800840A0008A900840A000853
:10336000AA008316031714089011831203138C11FB
:103370000317D30028083C39CB00243A0319032A49
:103380004B08043A0319C9294B08343A0319322A65
:1033900008005308031DFA295108213A031DF22998
:1033A000FF30D100831603172008A80022088312DB
:1033B000C70083162A088312C60083162108A900B5
:1033C0008312C2008317470884000008F1004608F2
:1033D000840071088000C70AC60AC20BE32983165D
:1033E0000830A00083160830A1008830A0008312A6
:1033F0002A2A0800083A031DFE2908005308103A3B
:1034000003190800080053081839031D252A51081C
:10341000063A031D0D2A2224242A5108663A031D68
:10342000132A2224242A5108053A031D192A8A2323
:10343000242A5108033A031D1E2A242A5108013A5E
:10344000031D232A242AC82C0800083A031D292A10
:103450000800080083160317A501C830A4008312D2
:10346000D101080083172A0884000008A000840AFC
:103470000008A100840A0008A200840A0008A30032
:10348000840A0008A400840A0008A500840A000831
:10349000A600840A0008A70083168830A000083020
:1034A000A100A40015128312D10120080319782A63
:1034B0002008013A0319892A2008023A0319952A9B
:1034C0002008803A03199D2A2008813A0319A92A65
:1034D0002008823A0319B52A20086039203A0319D6
:1034E000452C20086039403A031D442B442C080029
:1034F0002108013A0319942B2108053A0319812B5D
:103500002108093A0319D42B2108033A0319AD2BDA
:10351000442B2108013A0319AC2B21080B3A03195B
:10352000122C2108033A0319C52B2108013A03196B
:103530009B2B2108033A0319B42B2108083A0319DD
:10354000C72B2108063A0319BB2A2108003A0319A0
:10355000492B21080A3A0319FB2B2108003A0319C9
:10356000582B2108063A0319BB2A2108003A0319EF
:10357000632B442B08002308223A03197B2C2308D1
:10358000213A0319B32C1A308A0023080339CB3EA1
:1035900003188A0A8200442BCF2AE32A072B06301D
:1035A000D1000830C500F630AE001C30AF00F0246A
:1035B000C400A708031DE02A26022608031CC40035
:1035C000C40A222408000630D1000310220DDC2496
:1035D000AE000310220D013EDC24AF000230AE0726
:1035E0000318AF0AF024C4000230AE02031CAF037C
:1035F000A7080319FC2A022B440826020318022BF1
:103600002608C4000830C500C40A22240800663019
:10361000D1002408031D142B2508031D142B87300B
:10362000AE001D30AF00392B1D30AF008930AE0029
:10363000C8014F25AE0A2402031D222B4F25250267
:1036400003192A2BAE0AC80A8D302E02031C192B2F
:10365000D101442B06302202031C302BD101442B14
:10366000220DAF0048085525AE00AF0A4808552581
:10367000AF004F25C40026022608031CC4000830F2
:10368000C500C40A222408008316031718148312E5
:1036900008008316260884008312831752088000CE
:1036A000840A800183160230A500C830A4000800F7
:1036B0008316260884008001840A80010230A50058
:1036C000C830A40008000F302405013A0319722BFA
:1036D0000F302405023A031D442B031083161A18D9
:1036E0000314762B0310831619180314260884007C
:1036F0008001800D840A80010230A500C830A4003A
:1037000008000530D1002208CF008316A501C8307B
:10371000A4000800D101D0014F08831696000319B8
:10372000932B0230970008002208013A031D442B16
:10373000D2102A2208000F302405013A0319A82BC1
:103740000F302405023A031D442B83161A10AA2BAE
:10375000831619102A22080008002208013A031DC6
:10376000442BD2142A2208000F302405013A0319F1
:10377000C12B0F302405023A031D442B83161A1463
:10378000C32B831619142A220800442B0800831621
:1037900026088400831283175008800083160130A6
:1037A000A500C830A40008002208013C031C442BDB
:1037B0002208D0000319DF2B8316033097002A223A
:1037C000831603178830A800C830AA000830A90063
:1037D0004830AC00D030AE008830B000D830B200F5
:1037E0000830B1004830B400D830B6000E3099002F
:1037F0000E309A0008008316170883120339023A24
:103800000319442B24082B3E840083170008F10081
:10381000831626088400710880000130A500C83096
:10382000A40008008316170883120339033A031D06
:10383000442B831224082B3E840083172208800027
:103840002A22080083160317831726088400831290
:103850000317C0014008450203193A2CC40B312C50
:10386000392CF0248000C00A840AAE0F2A2CAF0A3B
:103870002A2CD10140088316A50040302406403987
:103880008838A4000800080008002008213A03191D
:103890005E2C2008223A0319CD2C2008233A031964
:1038A000CD2C2008A13A0319CD2C2008A23A0319E7
:1038B000CD2C2008A33A0319CD2C442B2108013A22
:1038C0000319CD2C2108023A0319CD2C2108033A03
:1038D0000319CD2C2108063A03197B2C2108093A3B
:1038E0000319CE2C21080A3A0319CD2C21080B3AD2
:1038F0000319D52C442B831203170630D10008304E
:10390000C5002308013A0319922C0310240DE62464
:10391000AE000310240D013EE624AF00F024C400E5
:10392000AE0AA82C2308023A0319A32C0310240D75
:10393000E624AE000310240D013EE624AF00F0247F
:10394000C400AE0AA82C2308033A0319442B08002C
:103950002708031DB02C2608440226080318C400BB
:10396000C40A222408000630D1000830C5001A30ED
:10397000AE001D30AF00F024C400A708031DC42C06
:1039800026022608031CC400C40A222408000800DA
:103990005108063A031922240800442B2130D10093
:1039A00083160317C830A0000800831603170030E1
:1039B000A500C830A4000800F1001C308A00E430E3
:1039C000710703188A0A820008341D34F1001C3084
:1039D0008A00EE30710703188A0A820031341D34E0
:1039E000831203172F088A002E0882001234013434
:1039F000003401340034003400340834D834043442
:103A000010341134003400340134023400340134F1
:103A1000093402342934003401340134043480344C
:103A200032340934043400340034023403340034B2
:103A300000340034093421340034013400340134BA
:103A400022341D34003407340534813403340834FF
:103A500000340A34073405340134033408340034A4
:103A60000A341D3406340034FF3409340134A134DF
:103A7000013419340134293408341534003426341F
:103A8000FF340034753408349534083481340234FA
:103A9000193401342934083491340234C034831287
:103AA00003172F088A002E088200F1000310F10D81
:103AB0006425CE00F10A6425F10071088A004E08E1
:103AC0002F0703188A0A82001D308A006B307107A5
:103AD00003188A0A82006F341D347B341D34873406
:103AE0001D348D341D34A1341D34CF341D34DB34EA
:103AF0001D34E5341D3487341D34F5341D34093448
:103B00001E3437341E3443341E344D341E340634D0
:103B100003340934043404340834143403344D3485
:103B200000346934003463340034723400346F3448
:103B30000034633400346834003469340034703441
:103B400000342E3403345034003469340034633488
:103B500000343134003436340034433400343734E4
:103B600000343634003435340034203400345534D5
:103B700000345334003442340034203400344C34A4
:103B800000344334003444340034203400344434AA
:103B90000034453400344D3400344F3400340C3498
:103BA000033456340034313400342E34003430348D
:103BB0000034303400340A3403344334003466347F
:103BC00000346734003431340034103403344E345C
:103BD00000346F3400347434003468340034693491
:103BE00000346E34003467340034143403344D34FC
:103BF00000346934003463340034723400346F3478
:103C00000034633400346834003469340034703470
:103C100000342E34033450340034693400346334B7
:103C20000034313400343634003443340034373413
:103C30000034363400343534003420340034553404
:103C400000345334003442340034203400344C34D3
:103C500000344334003444340034203400344434D9
:103C60000034453400344D3400344F3400340C34C7
:103C7000033456340034313400342E3400343034BC
:103C80000034303400340A340334433400346634AE
:103C900000346734003431340034103403344E348B
:103CA00000346F34003474340034683400346934C0
:0A3CB00000346E3400346734003431
:02400E00F63F7B
:00000001FF
